:020000000528D1
:06000A00831600308500A2
:100010000F308600831200308B0085010B210E21EA
:10002000861206130616861D1F28CD208C0B13285A
:100030000E210B21051085100511212113280B21FC
:100040000930E4200630F1200330FE200612861627
:100050000030D7200830E4200530F1200230FE20A7
:1000600086120617861D3C28CD208C0B32280515DC
:100070000E210B21212132280B210730E4200430EE
:10008000F1200130FE200F3003110E060319102855
:100090000E088000051D692805185C28851C692844
:1000A0000E309000B5200F308E00840A0408203AEC
:1000B000031D10288510672800309000B5200F30F0
:1000C0008E00840A0408203A031D1028051005112B
:1000D0000E280F308E00840A0408193A031D1028D8
:1000E0000E210408073E8900C920000803110806F4
:1000F000031D8228840A0408193A031D7128051477
:100100002B210E280E210408153E8900C920000865
:1001100003110806031D9428840A0408193A031DD4
:10012000832885142B210E280E210408003E890007
:10013000C920000803110806031DA428840A040826
:10014000193A031D952813210E2104080E3E89003B
:10015000C920000803110806031D0E28840A04089C
:10016000193A031DA5281A210E288B1300088800B0
:100170000408100789008316081555308900AA3035
:1001800089008814081EC2280812081183128B17D0
:10019000080083160814831208008D018D0A0D08CB
:1001A000163A0319D62800000000CE2808008F0058
:1001B000861DE228CD208C0BD8280F088E000B213D
:1001C0002121D8280B2108008F00061DEF28CD2003
:1001D0008C0BE5280F088E000B212121E5280B212F
:1001E00008008F00861CFC28CD208C0BF2280F08FD
:1001F0008E000B212121F2280B2108008F00061C04
:100200000929CD208C0BFF280F088E000B212121FE
:10021000FF280B2108007C308C0008000F308E0076
:1002200012308400080085191729851518298511B1
:100230002B210800051A1E2905161F2905122B213E
:1002400008008C0B242929298617CD208613CD2060
:1002500021298C0A08000A309100910B302933299A
:0A0260000B2121212D290B2108009C
:00000001FF
